:020000040000FA
:0600000068EF20F0120081
:020006001200E6
:06000800D5EF18F0120014
:02000E00C2909E
:040010009D9C1200A1
:04001400B46A1200B8
:0600180030EF19F01200A8
:02001E000500DB
:100020002A410000FE0800000200000028410000F4
:10003000FE0700000200000026410000FE0600004E
:100040000200000024410000FE0500000200000044
:0C00500022410000FE040000020000003D
:04005C00D9CFE6FF13
:10006000E1CFD9FF490EE126240EDB6A250EDB6ABB
:10007000260EDB6A270EDB6A280EDB6A9B8C8F0E4E
:10008000D3147009D36EFC0ED3140009D36E0F0184
:1000900048691F0E496FC9EC1DF0D9CFE6FFDACFD2
:1000A000E6FFA8EC13F0E552E552D950090FE66ED1
:1000B000000EDA20E66E1FEC09F0E552E552D95049
:1000C000190FE66E000EDA20E66ED9EC16F0E55256
:1000D000E5521AEC10F04FEC1BF0AAEC19F0FCEC16
:1000E0001BF0CDEC1CF097EC18F08CEC18F099ECB0
:1000F00009F0AAEC1AF0F6EC1CF080EC13F0000EFC
:10010000E66E0A0EE66ED950230FE66E000EDA2078
:10011000E66EFE0EE66E94EC12F0106E050EE15ED9
:100120001050210EF3CFDBFF220EF4CFDBFF210EA8
:10013000DBCF10F0220EDBCF11F00001800E111486
:100140000EE0D950210FE96EDACFEAFFFC0EEE186F
:1001500002E04EEF05F0FF0EED184EEF05F0230E16
:10016000DB50440A02E1E0EF04F0070A01E162D348
:10017000010A01E155D3030A01E14FD3010A01E16C
:1001800049D37F0A01E143D3010A01E13DD3030AC8
:1001900001E1D7D2010A01E115D1120A02E14EEFC5
:1001A00005F0030A07E0010A02E14EEF05F0070A35
:1001B0004EEF05F0240EDB6ADB50106E116A210E43
:1001C000DBCF12F0220EDBCF13F011501318E8AE84
:1001D00002D0133404D01250105C1350115803E2B3
:1001E000240EDB2AE9D7270EDB0402E10A0E05D034
:1001F000270EDB50020810E10B0EE66E09EC17F03B
:10020000E552000EE66E0A0EE66E060EE66E72EC23
:1002100017F0E552E552E55276EC18F0F3CF10F006
:10022000F4CF11F0070EF35C000EF45802E34EEF2A
:1002300005F013EC20F0D950330FE96EDACFEAFF66
:10024000000EEE6E0A0EED6E330EDBCFE9FF340EBC
:10025000DBCFEAFF100EEF6E330EDBCFE9FF340E7B
:10026000DBCFEAFFEE52EF6A330EDBCFE9FF340E4D
:10027000DBCFEAFF020EE926000EEA222B0EDBCFCF
:10028000EEFF2C0EDBCFEEFF2D0EDBCFEEFF2E0EA2
:10029000DBCFEEFF330EDBCFE9FF340EDBCFEAFF1F
:1002A000020EE926000EEA22040EE926000EEA22DA
:1002B0002F0EDBCFEEFF300EDBCFEEFF310EDBCFAC
:1002C000EEFF320EDBCFEEFF330EDBCFE9FF340E55
:1002D000DBCFEAFF020EE926000EEA22E9CF10F09A
:1002E000EACF11F0E9CFE6FFEACFE6FFBEEC15F06A
:1002F000E552E552330EDBCFE9FF340EDBCFEAFFE8
:100300000A0EE926000EEA22250EDBCFEEFF260EAE
:10031000DBCFEDFF330EDBCFE9FF340EDBCFEAFF9F
:100320000A0EE926000EEA22E9CF10F0EACF11F01A
:10033000E9CFE6FFEACFE6FFA6EC16F0E552E5527C
:10034000330EDBCFE9FF340EDBCFEAFF0C0EE926DC
:10035000000EEA22EF6A330EDBCFE9FF340EDBCF6B
:10036000EAFF0D0EE926000EEA22010EEF6E1D0EC9
:10037000DBCF10F01E0EDBCF11F00E0E1026000E9C
:100380001122210E10C0DBFF220E11C0DBFF330E45
:10039000DBCFE9FF340EDBCFEAFF0E0EE926000EBD
:1003A000EA22E9CF10F0EACF11F0E9CFE6FFEACF79
:1003B000E6FF1D0EDBCFE6FFFDEC17F0E552E55240
:1003C000E5525DD3D950370FE96EDACFEAFF000E60
:1003D000EE6E0A0EED6E240EDB6ADB50106E116AB3
:1003E000210EDBCF12F0220EDBCF13F0050E125ED2
:1003F000000E135A11501318E8AE02D0133404D073
:100400001250105C1350115803E2240EDB2AE5D77A
:10041000370EDBCFE9FF380EDBCFEAFF020EE9260D
:10042000000EEA22EF504D0801E0D1D0370EDBCFAD
:10043000E9FF380EDBCFEAFF020EE926000EEA22C2
:10044000010EE926000EEA22EF50500801E0BFD06D
:10045000370EDBCFE9FF380EDBCFEAFF050EE926CA
:10046000000EEA22290EEFCFDBFF370EDBCFE9FFCC
:10047000380EDBCFEAFF050EE926000EEA22010E58
:10048000E926000EEA222A0EEFCFDBFFD950290F12
:10049000E66E000EDA20E66EA6EC16F0E552E552A6
:1004A000290EDBCF06F02A0EDBCF07F0250E06C0A3
:1004B000DBFF260E07C0DBFFD950350FE96EDACF20
:1004C000EAFF000EEE6E0A0EED6E350EDBCFE9FF91
:1004D000360EDBCFEAFF080EEF6E350EDBCFE9FFFD
:1004E000360EDBCFEAFFEE52010EEF6E350EDBCF9C
:1004F000E9FF360EDBCFEAFF020EE926000EEA2204
:10050000420EEF6E350EDBCFE9FF360EDBCFEAFF92
:10051000020EE926000EEA22010EE926000EEA226A
:10052000480EEF6E350EDBCFE9FF360EDBCFEAFF6C
:10053000040EE926000EEA22010EEF6E050EF36EA0
:10054000210EF3CFDBFF220EDB6A210EDBCFE6FFAD
:10055000000EE66E0A0EE66E2CEC15F0E552E55242
:10056000E552D950350FE96EDACFEAFF000EEE6E94
:100570000A0EED6E350EDBCFE9FF360EDBCFEAFF5C
:10058000080EEF6E350EDBCFE9FF360EDBCFEAFF4C
:10059000EE52010EEF6E350EDBCFE9FF360EDBCFEC
:1005A000EAFF020EE926000EEA224E0EEF6E350E2D
:1005B000DBCFE9FF360EDBCFEAFF020EE926000EA5
:1005C000EA22010EE926000EEA22440E50D2370E2E
:1005D000DBCFE9FF380EDBCFEAFF020EE926000E83
:1005E000EA22EF504E0801E059D2370EDBCFE9FF87
:1005F000380EDBCFEAFF020EE926000EEA22010EDA
:10060000E926000EEA22EF50440801E047D2370EF7
:10061000DBCFE9FF380EDBCFEAFF050EE926000E3F
:10062000EA22020EE926000EEA222B0EEFCFDBFFB4
:10063000370EDBCFE9FF380EDBCFEAFF050EE926E8
:10064000000EEA22030EE926000EEA222C0EEFCF5E
:10065000DBFF370EDBCFE9FF380EDBCFEAFF050EFD
:10066000E926000EEA22040EE926000EEA222D0EEB
:10067000EFCFDBFF370EDBCFE9FF380EDBCFEAFF32
:10068000050EE926000EEA22050EE926000EEA22F2
:100690002E0EEFCFDBFF370EDBCFE9FF380EDBCFBF
:1006A000EAFF050EE926000EEA22060EE926000EF4
:1006B000EA222F0EEFCFDBFF370EDBCFE9FF380E3C
:1006C000DBCFEAFF050EE926000EEA22070EE92637
:1006D000000EEA22300EEFCFDBFF370EDBCFE9FF53
:1006E000380EDBCFEAFF050EE926000EEA22080EDF
:1006F000E926000EEA22310EEFCFDBFF370EDBCF0B
:10070000E9FF380EDBCFEAFF050EE926000EEA22EC
:10071000090EE926000EEA22320EEFCFDBFFD95098
:100720002B0FE66E000EDA20E66EBEEC15F0E552F9
:10073000E552010EF36E280EF3CFDBFF06EC1DF041
:10074000ADD113EC20F0D950390FE96EDACFEAFFC2
:10075000000EEE6E0A0EED6E390EDBCFE9FF3A0E9B
:10076000DBCFEAFFEE52E9CF10F0EACF11F0E9CF8C
:10077000E6FFEACFE6FFBEEC15F0E552E552390E92
:10078000DBCFE9FF3A0EDBCFEAFF090EE926000EC8
:10079000EA22E9CF10F0EACF11F0E9CFE6FFEACF85
:1007A000E6FFA6EC16F0E552E552240EDB6ADB50BC
:1007B000106E116A210EDBCF12F0220EDBCF13F088
:1007C0000C0E125E000E135A11501318E8AE02D030
:1007D000133404D01250105C1350115803E2240E4D
:1007E000DB2AE5D7390EDBCFE9FF3A0EDBCFEAFF94
:1007F0000C0EE926000EEA22EF50E66EF5EC19F039
:10080000E55207EC20F04AD1D9503B0F0BD0D9501C
:100810003D0F08D0D9503F0F05D0D950410F02D01D
:10082000D950430FE96EDACFEAFF000EEE6E0A0EE2
:10083000ED6E34D1D950450FE96EDACFEAFF000EE4
:10084000EE6E0A0EED6E450EDBCFE9FF460EDBCFF6
:10085000EAFFEE52E9CF10F0EACF11F0E9CFE6FF60
:10086000EACFE6FFBEEC15F0E552E552450EDBCFD0
:10087000E9FF460EDBCFEAFF0E0EE926000EEA2264
:10088000E9CF10F0EACF11F0E9CFE6FFEACFE6FFBB
:10089000BEEC15F0E552E552450EDBCFE9FF460E02
:1008A000DBCFEAFF090EE926000EEA22E9CF10F0BD
:1008B000EACF11F0E9CFE6FFEACFE6FFA6EC16F0AB
:1008C000E552E552450EDBCFE9FF460EDBCFEAFFEE
:1008D0000C0EE926000EEA22E9CF10F0EACF11F063
:1008E000E9CFE6FFEACFE6FFA6EC16F0E552E552C7
:1008F000450EDBCFE9FF460EDBCFEAFF180EE926F7
:10090000000EEA22E9CF10F0EACF11F0E9CFE6FFBE
:10091000EACFE6FFA6EC16F0E552E552100EE66EC1
:1009200009EC17F0E552450EDBCFE9FF460EDBCFB1
:10093000EAFF0E0EE926000EEA22E9CF10F0EACF18
:1009400011F0E9CFE6FFEACFE6FF040EE66E72ECA7
:1009500017F0E552E552E552450EDBCFE9FF460EB2
:10096000DBCFEAFF0E0EE926000EEA22040EE9268E
:10097000000EEA22E9CF10F0EACF11F0E9CFE6FF4E
:10098000EACFE6FF040EE66E72EC17F0E552E55290
:10099000E552450EDBCFE9FF460EDBCFEAFF0C0E3A
:1009A000E926000EEA22E9CF10F0EACF11F0E9CFF4
:1009B000E6FFEACFE6FF020EE66E72EC17F068D0B3
:1009C000D950470FE96EDACFEAFF000EEE6E0A0E3D
:1009D000ED6E470EDBCFE9FF480EDBCFEAFFEE52AC
:1009E000EF50110A5BE0160A59E0010A57E0050AC8
:1009F00053E0010A07E0030A51E0010A4FE1280E23
:100A0000DB6A4CD0D950350FE96EDACFEAFF000E21
:100A1000EE6E0A0EED6E350EDBCFE9FF360EDBCF44
:100A2000EAFF080EEF6E350EDBCFE9FF360EDBCFA7
:100A3000EAFFEE52010EEF6E350EDBCFE9FF360E08
:100A4000DBCFEAFF020EE926000EEA224D0EEF6E22
:100A5000350EDBCFE9FF360EDBCFEAFF020EE926CB
:100A6000000EEA22010EE926000EEA22500EEF6E79
:100A7000040EF36E210EF3CFDBFF220EDB6A210E94
:100A8000DBCFE6FF000EE66E0A0EE66E2CEC15F0EC
:100A9000E552E552E55202D0F6EC1CF0000EE66E8F
:100AA0000A0EE66ED950230FE66E000EDA20E66ECF
:100AB000FE0EE66E4BEC12F0106E050EE15E10506D
:100AC000210EF3CFDBFF220EF4CFDBFF210EDBCFB5
:100AD00010F0220EDBCF11F00001800E11140EE099
:100AE000D950210FE96EDACFEAFFFC0EEE1802E0D2
:100AF0007DEF00F0FF0EED187DEF00F0230EDB50D0
:100B00000C0A02E17DEF00F0070A01E169D3010A56
:100B100001E162D3470A01E156D3010A01E18FD214
:100B2000070A01E186D2010A01E1D4D1030A01E1F9
:100B3000C9D1010A01E115D10F0A14E0010A05E04B
:100B4000160A02E17DEF00F05FD3280EDB0402E01D
:100B50007DEF00F013EC20F0A0EC1BF0F6EC1CF0A5
:100B60007DEF00F0280EDB0402E07DEF00F013ECD7
:100B700020F0A9EC1BF0D950330FE96EDACFEAFF71
:100B8000000EEE6E0A0EED6E330EDBCFE9FF340E73
:100B9000DBCFEAFF100EEF6E330EDBCFE9FF340E32
:100BA000DBCFEAFFEE52EF6A330EDBCFE9FF340E04
:100BB000DBCFEAFF020EE926000EEA222B0EDBCF86
:100BC000EEFF2C0EDBCFEEFF2D0EDBCFEEFF2E0E59
:100BD000DBCFEEFF330EDBCFE9FF340EDBCFEAFFD6
:100BE000020EE926000EEA22040EE926000EEA2291
:100BF0002F0EDBCFEEFF300EDBCFEEFF310EDBCF63
:100C0000EEFF320EDBCFEEFF330EDBCFE9FF340E0B
:100C1000DBCFEAFF020EE926000EEA22E9CF10F050
:100C2000EACF11F0E9CFE6FFEACFE6FFBEEC15F020
:100C3000E552E552330EDBCFE9FF340EDBCFEAFF9E
:100C40000A0EE926000EEA22250EDBCFEEFF260E65
:100C5000DBCFEDFF330EDBCFE9FF340EDBCFEAFF56
:100C60000A0EE926000EEA22E9CF10F0EACF11F0D1
:100C7000E9CFE6FFEACFE6FFA6EC16F0E552E55233
:100C8000330EDBCFE9FF340EDBCFEAFF0C0EE92693
:100C9000000EEA22EF6A330EDBCFE9FF340EDBCF22
:100CA000EAFF0D0EE926000EEA22010EEF6E1D0E80
:100CB000DBCF10F01E0EDBCF11F00E0E1026000E53
:100CC0001122210E10C0DBFF220E11C0DBFF330EFC
:100CD000DBCFE9FF340EDBCFEAFF0E0EE926000E74
:100CE000EA22E9CF10F0EACF11F0E9CFE6FFEACF30
:100CF000E6FF1D0EDBCFE6FFFDEC17F0E552E552F7
:100D0000E552210EDBCFE6FF000EE66E0A0EE66E20
:100D10002CEC15F0E552E552E552330EDBCFE9FF3E
:100D2000340EDBCFEAFF0E0EE926000EEA22110E8A
:100D3000EF6E0F0EF36E210EF3CFDBFF220EDB6A98
:100D4000210EDBCFE6FF000EE66E0A0EE66E2CECFF
:100D500015F0E552E552E552270EDB6A06EC1DF070
:100D600037D2280EDB0402E07DEF00F013EC20F018
:100D7000DBEC1BF0D950330FE96EDACFEAFF000E3F
:100D8000EE6E0A0EED6E330EDBCFE9FF340EDBCFD5
:100D9000EAFF100EEF6E330EDBCFE9FF340EDBCF30
:100DA000EAFFEE52EF6A330EDBCFE9FF340EDBCF02
:100DB000EAFF020EE926000EEA222B0EDBCFEEFF41
:100DC0002C0EDBCFEEFF2D0EDBCFEEFF2E0EDBCF9A
:100DD000EEFF330EDBCFE9FF340EDBCFEAFF020E6E
:100DE000E926000EEA22040EE926000EEA222F0E62
:100DF000DBCFEEFF300EDBCFEEFF310EDBCFEEFFB1
:100E0000320EDBCFEEFF330EDBCFE9FF340EDBCF4C
:100E1000EAFF020EE926000EEA22E9CF10F0EACF3F
:100E200011F0E9CFE6FFEACFE6FFBEEC15F0E552A0
:100E3000E552330EDBCFE9FF340EDBCFEAFF0A0EBB
:100E4000E926000EEA22250EDBCFEEFF260EDBCFD1
:100E5000EDFF330EDBCFE9FF340EDBCFEAFF0A0EE6
:100E6000E926000EEA22E9CF10F0EACF11F0E9CF2F
:100E7000E6FFEACFE6FFA6EC16F0E552E552330EA8
:100E8000DBCFE9FF340EDBCFEAFF0C0EE926000EC4
:100E9000EA22EF6A330EDBCFE9FF340EDBCFEAFF45
:100EA0000D0EE926000EEA22010EEF6E330EDBCFA7
:100EB000E9FF340EDBCFEAFF0E0EE926000EEA2230
:100EC0000C0E6BD1280EDB0402E07DEF00F0E2ECAB
:100ED0001BF07ED1280EDB0402E07DEF00F013EC66
:100EE00020F0D950330FE96EDACFEAFF000EEE6E34
:100EF0000A0EED6E330EDBCFE9FF340EDBCFEAFFD7
:100F0000100EEF6E330EDBCFE9FF340EDBCFEAFFBE
:100F1000EE52EF6A330EDBCFE9FF340EDBCFEAFF90
:100F2000020EE926000EEA222B0EDBCFEEFF2C0E7E
:100F3000DBCFEEFF2D0EDBCFEEFF2E0EDBCFEEFF75
:100F4000330EDBCFE9FF340EDBCFEAFF020EE926DA
:100F5000000EEA22040EE926000EEA222F0EDBCF55
:100F6000EEFF300EDBCFEEFF310EDBCFEEFF320EA9
:100F7000DBCFEEFF330EDBCFE9FF340EDBCFEAFF32
:100F8000020EE926000EEA22E9CF10F0EACF11F0B6
:100F9000E9CFE6FFEACFE6FFBEEC15F0E552E552F9
:100FA000330EDBCFE9FF340EDBCFEAFF0A0EE92672
:100FB000000EEA22250EDBCFEEFF260EDBCFEDFF83
:100FC000330EDBCFE9FF340EDBCFEAFF0A0EE92652
:100FD000000EEA22E9CF10F0EACF11F0E9CFE6FFE8
:100FE000EACFE6FFA6EC16F0E552E552330EDBCF72
:100FF000E9FF340EDBCFEAFF0C0EE926000EEA22F1
:10100000EF6A330EDBCFE9FF340EDBCFEAFF0D0EC4
:10101000E926000EEA22010EEF6E330EDBCFE9FF68
:10102000340EDBCFEAFF0E0EE926000EEA220E0E8A
:10103000B4D0280EDB0402E07DEF00F0C9D0280E0A
:10104000DB0402E07DEF00F013EC20F0D950330F09
:10105000E96EDACFEAFF000EEE6E0A0EED6E330E89
:10106000DBCFE9FF340EDBCFEAFF100EEF6E330E5D
:10107000DBCFE9FF340EDBCFEAFFEE52EF6A330E2F
:10108000DBCFE9FF340EDBCFEAFF020EE926000ECC
:10109000EA222B0EDBCFEEFF2C0EDBCFEEFF2D0E68
:1010A000DBCFEEFF2E0EDBCFEEFF330EDBCFE9FF03
:1010B000340EDBCFEAFF020EE926000EEA22040E10
:1010C000E926000EEA222F0EDBCFEEFF300EDBCF3B
:1010D000EEFF310EDBCFEEFF320EDBCFEEFF330E35
:1010E000DBCFE9FF340EDBCFEAFF020EE926000E6C
:1010F000EA22E9CF10F0EACF11F0E9CFE6FFEACF1C
:10110000E6FFBEEC15F0E552E552330EDBCFE9FF0A
:10111000340EDBCFEAFF0A0EE926000EEA22250E86
:10112000DBCFEEFF260EDBCFEDFF330EDBCFE9FF8B
:10113000340EDBCFEAFF0A0EE926000EEA22E9CFE1
:1011400010F0EACF11F0E9CFE6FFEACFE6FFA6EC18
:1011500016F0E552E552330EDBCFE9FF340EDBCF5C
:10116000EAFF0C0EE926000EEA22EF6A330EDBCF0F
:10117000E9FF340EDBCFEAFF0D0EE926000EEA226E
:10118000010EEF6E330EDBCFE9FF340EDBCFEAFF4B
:101190000E0EE926000EEA220D0EEF6E0F0EF36E14
:1011A000210EF3CFDBFF220EDB6A210EDBCFE6FF41
:1011B000000EE66E0A0EE66E2CEC15F0E552E552D6
:1011C000E5527DEF00F0280EDB0402E07DEF00F039
:1011D00007EC20F07DEF00F009EC20F07DEF00F04F
:1011E000270EDB50020807E0270EDB0404E125ECA4
:1011F0001BF0020E03D0FBEC1AF0010EF36E270E6B
:10120000F3CFDBFF7DEF00F0240EDB6ADB50106EC6
:10121000116A210EDBCF12F0220EDBCF13F011503A
:101220001318E8AE02D0133404D01250105C1350DF
:0E123000115802E37DEF00F0240EDB2AE7D711
:02123E00D9CF06
:10124000E6FFE1CFD9FFFD0EDBCFFEF2FE0EDBCFD6
:10125000FFF2FEC2E9FFFFC2EAFF000EEE6E0B0EC8
:10126000ED6EFEC2E9FFFFC2EAFF020EEB6A030E5B
:10127000EB6AFEC2E9FFFFC2EAFF060EE926000E96
:10128000EA22EF6AFEC2E9FFFFC2EAFF040EE92686
:10129000000EEA22050EEF6EFEC2E9FFFFC2EAFF72
:1012A000070EE926000EEA22EF6AFEC2E9FFFFC23E
:1012B000EAFF050EE926000EEA22EF6AFEC2E9FF08
:1012C000FFC2EAFF090EE926000EEA22EF6AFEC21B
:1012D000E9FFFFC2EAFF0B0EE926000EEA22EF6AE1
:1012E000FEC2E9FFFFC2EAFF0C0EE926000EEA2269
:1012F000EF6AFEC2E9FFFFC2EAFF0F0EE926000E09
:10130000EA22EF6AFEC2E9FFFFC2EAFF0D0EE926FC
:10131000000EEA22EF6AFEC2E9FFFFC2EAFF0E0EEC
:10132000E926000EEA22220EEF6EE552E7CFD9FF42
:101330001200FEC2E9FFFFC2EAFF0F0EE926000E0F
:10134000EA22110EEF6E94869488C76AC66AC56A4F
:10135000F00EC6140809C66E630EC86EC78EC68A24
:101360001200D9CFE6FFE1CFD9FF020EE126FD0E34
:10137000DB506FE0DE6ADD6ADECF10F0DDCF11F00A
:10138000FD0EDB50000111AE02D0D89003D0105CEE
:10139000000E115826E2FB0EDBCF12F0FC0EDBCF65
:1013A00013F0DE501224E96EDD501320EA6EEF5088
:1013B000E66EDECF10F0DDCF11F0FEC2E9FFFFC216
:1013C000EAFF1050EE24E76E1150EE20EA6EE7CFF0
:1013D000E9FFE552E750EF6EDF2A010ECDE3DB2A8D
:1013E000CBD7FD0EDB50E66EFEC2E9FFFFC2EAFF7F
:1013F000020EE926000EEA22E552E750EE6EED6A93
:10140000FEC2E9FFFFC2EAFF0D0EE926000EEA2246
:10141000FE0EDBCFEFFFFEC2E9FFFFC2EAFF050EC3
:10142000E926000EEA22EF6AFEC2E9FFFFC2EAFFE8
:10143000040EE926000EEA22090EEF6EFEC2E9FF55
:10144000FFC2EAFF0E0EE926000EEA22200EEF6E22
:10145000C580020EE15C02E2E16AE552E16EE5520E
:10146000E7CFD9FF1200D9CFE6FFE1CFD9FFFD0EBC
:10147000DB5038E0FD0EDB50E66EFEC2E9FFFFC236
:10148000EAFF020EE926000EEA22E552E750EE6E70
:10149000ED6AFEC2E9FFFFC2EAFF0D0EE926000E6B
:1014A000EA22FE0EDBCFEFFFFEC2E9FFFFC2EAFF3A
:1014B000050EE926000EEA22EF6AFEC2E9FFFFC22E
:1014C000EAFF040EE926000EEA22090EEF6EFEC2C4
:1014D000E9FFFFC2EAFF0E0EE926000EEA22210E06
:1014E000EF6EC580E552E7CFD9FF1200D9CFE6FFF6
:1014F000E1CFD9FFFEC2E9FFFFC2EAFF0F0EE926E6
:10150000000EEA22100EEF6E94869488FE0EDB50D9
:10151000E824C86EC76AC66AC56AF00EC6140E090A
:10152000C66EC78EC580C68AE552E7CFD9FF1200C6
:10153000FEC2E9FFFFC2EAFF0F0EEB50110802E105
:10154000ACEF0AF0FEC2E9FFFFC2EAFF0F0EEB505C
:10155000100801E1E4D91200FEC2E9FFFFC2EAFF70
:101560000E0EEB50200801E09DD0FEC2E9FFFFC245
:10157000EAFF040EEB500B0A19E0020A04E00C0A21
:1015800001E18FD01200FEC2E9FFFFC2EAFF040EA4
:10159000E926000EEA220B0EEF6EFEC2E9FFFFC243
:1015A000EAFF0D0EEB50E824C96E1200C5BC58D0FE
:1015B000FEC2E9FFFFC2EAFF050EEB50106E116A92
:1015C000020EE926000EEA22EECF12F0EFCF13F062
:1015D00011501318E8AE02D0133404D01250105C2E
:1015E000135011581BE2FEC2E9FFFFC2EAFF050ECD
:1015F000EB50116AE850EE24E76E1150EE20EA6ECF
:10160000E7CFE9FFEF50C96EFEC2E9FFFFC2EAFF74
:10161000050EE926000EEA22EF2A1200FEC2E9FFBB
:10162000FFC2EAFF040EE926000EEA22050EEF6E65
:10163000C584FEC2E9FFFFC2EAFF0E0EE926000ED6
:10164000EA22220EEF6E000EE66EE66A2B0EE66EC2
:10165000E66A77EC12F0E552E552E552E5521200E7
:10166000FEC2E9FFFFC2EAFF040EE926000EEA22ED
:10167000050EEF6EC584FEC2E9FFFFC2EAFF0E0E43
:10168000E926000EEA22220EEF6E000EE66EE66AF2
:101690002C0EE66EE66A77EC12F0E552E552E55262
:1016A000E5521200FEC2E9FFFFC2EAFF0E0EEB5048
:1016B000210801E0D7D0FEC2E9FFFFC2EAFF040E15
:1016C000EB500D0A01E19FD0010A01E190D00B0A15
:1016D00040E00C0A1AE0020A04E00C0A01E1C2D060
:1016E0001200FEC2E9FFFFC2EAFF040EE926000E67
:1016F000EA220B0EEF6EFEC2E9FFFFC2EAFF0D0EFB
:10170000EB50E8240109C96E1200C5AC70D0FEC2CE
:10171000E9FFFFC2EAFF040EE926000EEA22050EE9
:10172000EF6EC584FEC2E9FFFFC2EAFF0E0EE92696
:10173000000EEA22220EEF6E000EE66EE66A2E0E14
:10174000E66EE66A77EC12F0E552E552E552E552B4
:101750001200FEC2E9FFFFC2EAFF050EEB50116A5C
:10176000E850EE24E76E1150EE20EA6EE7CFE9FF75
:10177000C9CFEFFFFEC2E9FFFFC2EAFF050EE9266F
:10178000000EEA22EF2AFEC2E9FFFFC2EAFF050EC1
:10179000EB50106E116A020EE926000EEA22EECF1F
:1017A00012F0EFCF13F011501318E8AE02D013343B
:1017B00004D01250105C135011580CE2FEC2E9FF25
:1017C000FFC2EAFF040EE926000EEA220C0EEF6EBD
:1017D000C59A0BD0FEC2E9FFFFC2EAFF040EE9265C
:1017E000000EEA220D0EEF6EC58AC5881200FEC2F9
:1017F000E9FFFFC2EAFF040EE926000EEA22070E07
:10180000EF6EC5861200FEC2E9FFFFC2EAFF040EBA
:10181000E926000EEA22050EEF6EC584FEC2E9FF3E
:10182000FFC2EAFF0E0EE926000EEA22220EEF6E3C
:10183000FEC2E9FFFFC2EAFFEECFE6FFEFCFE6FF11
:101840002D0EE66EFEC2E9FFFFC2EAFF020EE92698
:10185000000EEA22EF50E66E77EC12F0E552E55208
:10186000E552E5521200D9CFE6FFE1CFD9FFFEC223
:10187000E9FFFFC2EAFF060EE926000EEA22010E8A
:10188000EF6EFEC2E9FFFFC2EAFF020EEB6A030E33
:10189000EB6AFE0EDB5035E0C7AA1DD0FEC2E9FFA1
:1018A000FFC2EAFF040EE926000EEA22050EEF6EE3
:1018B000FEC2E9FFFFC2EAFF080EE926000EEA2297
:1018C000EF2AFEC2E9FFFFC2EAFF070EE926000E7B
:1018D000EA22050E1FD0C7A40AD0FEC2E9FFFFC24C
:1018E000EAFF040EE926000EEA22080E13D0FEC21B
:1018F000E9FFFFC2EAFF040EE926000EEA22070E06
:1019000009D0FEC2E9FFFFC2EAFF040EE926000E7D
:10191000EA22060EEF6EE552E7CFD9FF1200D9CFCB
:10192000E6FFE1CFD9FF090EE126010EDB6A020EC8
:10193000DB6A030EDB6A040EDB6A080EDB6AC6ACE8
:1019400023D0C69CFEC2E9FFFFC2EAFF040EE926CF
:10195000000EEA22050EEF6E010EF36E040EF3CFB9
:10196000DBFFFEC2E9FFFFC2EAFF080EE926000E18
:10197000EA22EF2AFEC2E9FFFFC2EAFF070EE926CC
:10198000000EEA22040EEF6EC7A005D0C950DF6E2C
:10199000DE52010EDD6E040EDB5001E01FD2FEC2EE
:1019A000E9FFFFC2EAFF040EEB50070A01E15BD139
:1019B0000F0A6CE00E0A14E0030A01E00FD2C7A67A
:1019C0000DD2010EDBCFE6FF4EDFE552FEC2E9FF8E
:1019D000FFC2EAFF040EEB50080801E0FFD137D048
:1019E000C7A810D0FEC2E9FFFFC2EAFF060EE92633
:1019F000000EEA22EF2A010EDB5001E1E5D1C7AA71
:101A000084D1CFD1010EDB5001E1E8D1FEC2E9FF64
:101A1000FFC2EAFF060EE926000EEA22EF2AC7BA45
:101A200018D0C7B40AD0FEC2E9FFFFC2EAFF040E15
:101A3000E926000EEA22070ED0D1FEC2E9FFFFC25E
:101A4000EAFF040EE926000EEA22080EEF6E030EEE
:101A5000A6D1FEC2E9FFFFC2EAFF080EE926000E8A
:101A6000EA22EF2AFEC2E9FFFFC2EAFF040EE926DE
:101A7000000EEA22050EEF6EFEC2E9FFFFC2EAFF8A
:101A8000070EE926000EEA22060EA7D1FEC2E9FFE4
:101A9000FFC2EAFF0B0EEB50000901E07BD046ECE1
:101AA00013F0080EF3CFDBFFDB502A081BE0C968F8
:101AB000FEC2E9FFFFC2EAFF050EE926000EEA2298
:101AC000010EEF6EFEC2E9FFFFC2EAFF0B0EE92630
:101AD000000EEA22010EEF6EFEC2E9FFFFC2EAFF2E
:101AE0000C0E52D0FEC2E9FFFFC2EAFFEECFE6FFC6
:101AF000EFCFE6FFFEC2E9FFFFC2EAFF0A0EEB509E
:101B0000E66EE66AFE0EE66E26EC13F0126E050E29
:101B1000E15E1250F4CF11F0FEC2E9FFFFC2EAFF0E
:101B2000020EF3CFEBFF030E11C0EBFFFEC2E9FF85
:101B3000FFC2EAFF020EE926000EEA22EECF10F005
:101B4000EFCF11F0113401E349D110500008000E1D
:101B5000115401E343D1FEC2E9FFFFC2EAFFEE5098
:101B6000EFCFEAFFE96EEF50C96EFEC2E9FFFFC298
:101B7000EAFF050EE926000EEA22010EEF6EFEC214
:101B8000E9FFFFC2EAFF0B0EE926000EEA22010E72
:101B9000EF6E5AD0FEC2E9FFFFC2EAFF0C0EEB5017
:101BA00000091CE0FEC2E9FFFFC2EAFF050EEB5090
:101BB000106E090EEB50105C02E2C9683BD0FEC209
:101BC000E9FFFFC2EAFF0B0EE926000EEA22EF6AE8
:101BD000FEC2E9FFFFC2EAFF0C0E40D0FEC2E9FFE1
:101BE000FFC2EAFF050EEB50106E116A020EE926E5
:101BF000000EEA22EECF12F0EFCF13F011501318BF
:101C0000E8AE02D0133404D01250105C13501158B7
:101C100020E2FEC2E9FFFFC2EAFF050EEB50116AA7
:101C2000E850EE24E76E1150EE20EA6EE7CFE9FFB0
:101C3000EF50C96EFEC2E9FFFFC2EAFF050EE926BA
:101C4000000EEA22EF2A010EF36E020EF3CFDBFF45
:101C5000C5D0FEC2E9FFFFC2EAFF0B0EE926000E67
:101C6000EA22EF6AB1D0C7A856D0FEC2E9FFFFC290
:101C7000EAFF060EE926000EEA22EF2A010EDB50EB
:101C800044E0C7AA25D0FEC2E9FFFFC2EAFFEECFBB
:101C900010F0EFCF11F0FEC2E9FFFFC2EAFF020E23
:101CA000E926000EEA221050EE24E76E1150EE20D5
:101CB000EA6EE7CFE9FFDFCFEFFFFEC2E9FFFFC229
:101CC000EAFF020EE926000EEA22EE2AEF221DD0DC
:101CD000FEC2E9FFFFC2EAFF080EE926000EEA2273
:101CE000EF2AFEC2E9FFFFC2EAFF070EE926000E57
:101CF000EA22060EEF6EFEC2E9FFFFC2EAFF040E03
:101D0000E926000EEA22050E5ED0010EF36E030EE8
:101D1000F3CFDBFF59D0010EDB5060E0FEC2E9FFDC
:101D2000FFC2EAFF060EE926000EEA22EF2AC7AA42
:101D300025D0FEC2E9FFFFC2EAFFEECF10F0EFCFE1
:101D400011F0FEC2E9FFFFC2EAFF020EE926000E13
:101D5000EA221050EE24E76E1150EE20EA6EE7CF33
:101D6000E9FFDFCFEFFFFEC2E9FFFFC2EAFF020E8D
:101D7000E926000EEA22EE2AEF2230D0C7A411D0C5
:101D8000FEC2E9FFFFC2EAFF040EE926000EEA22C6
:101D9000080EEF6E010EF36E030EF3CFDBFFC96E7C
:101DA0001DD0FEC2E9FFFFC2EAFF080EE926000EC1
:101DB000EA22EF2AFEC2E9FFFFC2EAFF070EE92688
:101DC000000EEA22060EEF6EFEC2E9FFFFC2EAFF36
:101DD000040EE926000EEA22050EEF6E010EDB501E
:101DE00003E1020EDB5002E0C6A8C688FEC2E9FF8E
:101DF000FFC2EAFF020EE926000EEA22EECF10F043
:101E0000EFCF11F0113425E21050FC08000E1154F0
:101E100020E2030EDB501DE1FEC2E9FFFFC2EAFF34
:101E2000040EE926000EEA22050EEF6EFEC2E9FF5F
:101E3000FFC2EAFF080EE926000EEA22EF2AFEC2E0
:101E4000E9FFFFC2EAFF070EE926000EEA22070EAD
:101E5000EF6E030EDB506DE0FEC2E9FFFFC2EAFF4A
:101E6000020EE926000EEA22EECF10F0EFCF11F0BD
:101E70001006115AFEC2E9FFFFC2EAFF1050EE241D
:101E8000E76E1150EE20EA6EE7CFE9FFEF50E66E05
:101E9000FEC2E9FFFFC2EAFF090EE926000EEA22B0
:101EA000E552E750EF6EFEC2E9FFFFC2EAFF060E01
:101EB000EB50E66EEECF10F0EFCF11F0FEC2E9FF6F
:101EC000FFC2EAFF020EE926000EEA221050EE24BD
:101ED000E76E1150EE20EA6EE7CFE9FFE552E750DA
:101EE000EF6EFEC2E9FFFFC2EAFFEECFE6FFEFCFE3
:101EF000E6FF290EE66EFEC2E9FFFFC2EAFF020E10
:101F0000E926000EEA22EECF10F0EFCF11F0010E1D
:101F10001024E66E77EC12F0E552E552E552E552F8
:101F2000FEC2E9FFFFC2EAFF020EEB6A030EEB6A94
:101F300038D0FEC2E9FFFFC2EAFF080EEB50106E78
:101F4000010E105C2EE3FEC2E9FFFFC2EAFF080E9D
:101F5000EB50E76E050EE7CFDBFF070EEB50E76EA9
:101F6000060EE7CFDBFFEB50E76E070EE7CFDBFF98
:101F7000D950050FE66E000EDA20E66E280EE66EEA
:101F8000030EE66E77EC12F0E552E552E552E552AB
:101F9000FEC2E9FFFFC2EAFF080EE926000EEA22B0
:101FA000EF6A090EE15C02E2E16AE552E16EE55298
:101FB000E7CFD9FF1200FEC2E9FFFFC2EAFF0E0E13
:0A1FC000EB50220801E1000C010CB7
:061FCA00D9CFE6FFE1CFD4
:101FD000D9FFE652FD0EDBCFE9FFFE0EDBCFEAFFB5
:101FE0000A0EE926000EEA22EF6AFD0EDBCFE9FFBA
:101FF000FE0EDBCFEAFF0B0EE926000EEA22EF6AA7
:10200000DF6A020EDF5C11E2FD0EDBCFE9FFFE0EA0
:10201000DBCFEAFFDF50050DE950F324E96EEA500B
:10202000F420EA6EEF6ADF2AECD7E552E552E7CFFB
:10203000D9FF12000001906B000E636F090E646FF0
:10204000000E686F080E696F000E6F6F070E706FDD
:10205000000E746F060E756F000E7B6F050E7C6FA1
:10206000000E806F040E816F000E876F030E886F65
:10207000000E8C6F020E8D6F600EE66E000EE66E27
:10208000A4DFE552E5526C0EE66E000EE66E9DDFB3
:10209000E552E552780EE66E000EE66E96DFE552EA
:1020A000E552840EE66E000EE66E8FDFE552E552D5
:1020B0001200D9CFE6FFE1CFD9FF050EE126FC0ED5
:1020C000DB50E66ED950030FE96EDACFEAFFE55236
:1020D000E750EE6EED6AFD0EDBCFE9FFFE0EDBCFC3
:1020E000EAFF0A0EE926000EEA22EFCFDFFFFD0E1F
:1020F000DBCFE9FFFE0EDBCFEAFFE9CF12F0EACF3C
:1021000013F0DF50050DE950F324106EEA50F4206F
:10211000116E010E10C0DBFF020E11C0DBFF010EBD
:10212000DBCFE9FF020EDBCFEAFFEF5003E0F368FD
:10213000F4685AD0010EDBCFE9FF020EDBCFEAFFD5
:10214000EE52FC0EDBCFEFFF010EDBCFE9FF020EFC
:10215000DBCFEAFFE926000EEA22FB0EDBCFEFFF22
:10216000030EDBCFE6FF040EDBCFE6FFF90EDBCF7D
:10217000E6FFFA0EDBCFE6FF010EDBCFE9FF020E32
:10218000DBCFEAFF030EE926000EEA22EECFE6FFE0
:10219000EFCFE6FFE1EC1EF0106E060EE15E105090
:1021A000FD0EDBCFE9FFFE0EDBCFEAFF0A0EE926CC
:1021B000000EEA22EF28010BE66EFD0EDBCFE9FFF1
:1021C000FE0EDBCFEAFF0A0EE926000EEA22E552F8
:1021D000E750EF6E010EDBCFE9FF020EDBCFEAFF27
:1021E000010EEF6EF36EF46A050EE15C02E2E16A45
:1021F000E552E16EE552E7CFD9FF1200D9CFE6FFF5
:10220000E1CFD9FF050EE126FD0EDBCFE9FFFE0E83
:10221000DBCFEAFF0B0EE926000EEA22EFCFDFFF4D
:10222000FD0EDBCFE9FFFE0EDBCFEAFFE9CF12F0B8
:10223000EACF13F0DF50050DE950F324106EEA5099
:10224000F420116E010E10C0DBFF020E11C0DBFF87
:10225000010EDBCFE9FF020EDBCFEAFFEF0401E066
:1022600082D0010EDBCFE9FF020EDBCFEAFFEE5298
:10227000EFCF10F0FC0EDB50D880105402E2FD0EC0
:1022800073D0010EDBCFE9FF020EDBCFEAFFEE5287
:10229000EF50E66ED950030FE96EDACFEAFFE55250
:1022A000E750EE6EED6A030EDBCFE6FF040EDBCFE8
:1022B000E6FF010EDBCFE9FF020EDBCFEAFF030EE4
:1022C000E926000EEA22EECFE6FFEFCFE6FFF80E9A
:1022D000DBCFE6FFF90EDBCFE6FFE1EC1EF0106E80
:1022E000060EE15E1050FD0EDBCFE9FFFE0EDBCFE8
:1022F000EAFF0B0EE926000EEA22EF28010BE66E3C
:10230000FD0EDBCFE9FFFE0EDBCFEAFF0B0EE92669
:10231000000EEA22E552E750EF6E010EDBCFE9FF37
:10232000020EDBCFEAFFE926000EEA22EF50E66E4E
:10233000FA0EDBCFE9FFFB0EDBCFEAFFE552E750F9
:10234000EF6E010EDBCFE9FF020EDBCFEAFFEF6A93
:10235000030EDBCF10F0040EDBCF11F010C0F3FF43
:1023600011C0F4FF03D0FC0EF36EF468050EE15CBF
:1023700002E2E16AE552E16EE552E7CFD9FF1200D1
:10238000D9CFE6FFE1CFD9FF030EE126FD0EDBCF6B
:10239000E9FFFE0EDBCFEAFF0B0EE926000EEA2274
:1023A000EFCFDFFFFD0EDBCFE9FFFE0EDBCFEAFF55
:1023B000DF50050DE950F324106EEA50F420116E41
:1023C000010E10C0DBFF020E11C0DBFF010EDBCFE0
:1023D000E9FF020EDBCFEAFFEF040BE1010EDBCFDA
:1023E000E9FF020EDBCFEAFFE926000EEA22EF50FA
:1023F00001D0000E106E030EE15C02E2E16AE552CC
:10240000E16E1050E552E7CFD9FF1200D9CFE6FFB9
:10241000E1CFD9FFFD0EDBCFE9FFFE0EDBCFEAFFF8
:10242000E9CF10F0EACF11F0FD0EDBCFE9FFFE0E91
:10243000DBCFEAFF0B0EE926000EEA22EF50050D76
:102440001050F324E96E1150F420EA6EEF50E5527B
:10245000E7CFD9FF1200D38E03001200D9CFE6FFD9
:10246000E1CFD9FFFB0EDBCFE6FFFC0EDBCFE6FFB3
:10247000FD0EDBCFE6FFFE0EDBCFE6FF600EE66E65
:10248000000EE66E16DE106E060EE15E1050E5528E
:10249000E7CFD9FF1200D9CFE6FFE1CFD9FFFA0E7F
:1024A000DBCFE6FFFB0EDBCFE6FFFC0EDBCFE6FF6C
:1024B000FD0EDBCFE6FFFE0EDBCFE6FF600EE66E25
:1024C000000EE66E9BDE106E070EE15E1050E552C8
:1024D000E7CFD9FF1200600EE66E000EE66E50DF09
:1024E000E552E552116AF36E11C0F4FF1200D9CF24
:1024F000E6FFE1CFD9FFFB0EDBCFE6FFFC0EDBCF23
:10250000E6FFFD0EDBCFE6FFFE0EDBCFE6FF6C0E37
:10251000E66E000EE66ECDDD106E060EE15E10502A
:10252000E552E7CFD9FF1200D9CFE6FFE1CFD9FFBF
:10253000FA0EDBCFE6FFFB0EDBCFE6FFFC0EDBCFB8
:10254000E6FFFD0EDBCFE6FFFE0EDBCFE6FF6C0EF7
:10255000E66E000EE66E52DE106E070EE15E105063
:10256000E552E7CFD9FF12006C0EE66E000EE66E64
:1025700007DFE552E552116AF36E11C0F4FF120055
:10258000D9CFE6FFE1CFD9FFFB0EDBCFE6FFFC0E94
:10259000DBCFE6FFFD0EDBCFE6FFFE0EDBCFE6FF77
:1025A000780EE66E000EE66E84DD106E060EE15EBD
:1025B0001050E552E7CFD9FF1200D9CFE6FFE1CFA7
:1025C000D9FFFA0EDBCFE6FFFB0EDBCFE6FFFC0EFA
:1025D000DBCFE6FFFD0EDBCFE6FFFE0EDBCFE6FF37
:1025E000780EE66E000EE66E09DE106E070EE15EF6
:1025F0001050E552E7CFD9FF1200780EE66E000EBC
:10260000E66EBEDEE552E552116AF36E11C0F4FFCC
:102610001200D9CFE6FFE1CFD9FFFB0EDBCFE6FFFB
:10262000FC0EDBCFE6FFFD0EDBCFE6FFFE0EDBCFC1
:10263000E6FF840EE66E000EE66E3BDD106E060EC3
:10264000E15E1050E552E7CFD9FF1200D9CFE6FF87
:10265000E1CFD9FFFA0EDBCFE6FFFB0EDBCFE6FFC3
:10266000FC0EDBCFE6FFFD0EDBCFE6FFFE0EDBCF81
:10267000E6FF840EE66E000EE66EC0DD106E070EFD
:10268000E15E1050E552E7CFD9FF1200840EE66EEE
:10269000000EE66E75DEE552E552116AF36E11C06A
:1026A000F4FF12000001905101E11200B7EC18F0A4
:1026B000F3CF10F0F4CF11F0F350F41001E012005A
:1026C0009BEC18F0F3CF10F0F4CF11F0F350F410AE
:1026D00001E112006C0EE66E000EE66E97DEE5522A
:1026E000E552000901E01200600EE66E000EE66E93
:1026F0008DDEE552E552000901E012002BEF12F0E9
:10270000C3EC18F0F3CF10F0F4CF11F0F350F41045
:1027100001E112000001010E906F6C0EE66E000EDA
:10272000E66E74DEE552E552000909E1600EE66EE0
:10273000000EE66E6BDEE552E552000903E0000193
:10274000906B12000A0EE66E48EC20F0E552E5D7D9
:10275000D9CFE6FFE1CFD9FF93809392949A8A90E4
:102760008A928B9AFD0EDBCF9BF0FE0EDBCF9CF0A6
:102770009BC0E9FF9CC0EAFF050EE926000EEA2295
:10278000EF6A9BC0E9FF9CC0EAFF060EE926000E37
:10279000EA22EF6A9BC0E9FF9CC0EAFF070EE92628
:1027A000000EEA220A0EEF6E9BC0E9FF9CC0EAFF12
:1027B000030EE926000EEA22000EEE6E010EED6E0B
:1027C0009BC0E9FF9CC0EAFF030EE926000EEA2247
:1027D000EECF9DF0EDCF9EF0E552E7CFD9FF12008E
:1027E000D9CFE6FFE1CFD9FFFE0EDB507E0823E113
:1027F0009BC0E9FF9CC0EAFF050EE926000EEA2215
:10280000EF6A9BC0E9FF9CC0EAFF060EE926000EB6
:10281000EA22EF6A9BC0E9FF9CC0EAFF7E0EEF6EE2
:102820009BC0E9FF9CC0EAFF070EE926000EEA22E2
:102830000B0EEF6EA4D09BC0E9FF9CC0EAFF070E11
:10284000EB500F0A01E181D0010A2EE0020A1AE0E2
:10285000070A02E0010A93D09BC0E9FF9CC0EAFF8F
:10286000EE52010EE926000EEA22FE0EDBCFEFFF4C
:102870009BC0E9FF9CC0EAFF070EE926000EEA2292
:102880000C0E7CD09BC0E9FF9CC0EAFFEE52FE0E0E
:10289000DBCFEFFF9BC0E9FF9CC0EAFF070EE926F4
:1028A000000EEA220E0E6AD09BC0E9FF9CC0EAFF30
:1028B000050EEB50106EEE52EECF11F0EFCF12F08E
:1028C0001150105C000E125423E29BC0E9FF9CC023
:1028D000EAFF050EEB500001EA6A9D25E96E9E5164
:1028E000EA22FE0EDBCFEFFF9BC0E9FF9CC0EAFFB0
:1028F000060EE926000EEA22FE0EDB50EF269BC0F4
:10290000E9FF9CC0EAFF050EE926000EEA22EF2A45
:102910009BC0E9FF9CC0EAFF050EEB50106E116AE8
:10292000EE52EECF12F0EFCF13F01250101827E155
:102930001350111824E19BC0E9FF9CC0EAFF070E69
:10294000E926000EEA220F0E19D09BC0E9FF9CC0B9
:10295000EAFF060EE926000EEA22EF28E86C106E68
:10296000FE0EDB50105C01E10ED89BC0E9FF9CC05D
:10297000EAFF070EE926000EEA220A0EEF6EE55284
:10298000E7CFD9FF1200D9CFE6FFE1CFD9FFE6525A
:102990009DC0E9FF9EC0EAFFEF508A0A40E01F0A8F
:1029A00038E0340A30E0360A28E0060A20E0030A5C
:1029B00018E0190A10E01B0A08E0180A48E19DC057
:1029C000E6FF9EC0E6FF3C0E2FD09DC0E6FF9EC0F6
:1029D000E6FF3D0E29D09DC0E6FF9EC0E6FF3E0EFD
:1029E00023D09DC0E6FF9EC0E6FF3F0E1DD09DC0D8
:1029F000E6FF9EC0E6FF400E17D09DC0E6FF9EC0DA
:102A0000E6FF410E11D09DC0E6FF9EC0E6FF420EDC
:102A10000BD09DC0E6FF9EC0E6FF430E05D09DC0D3
:102A2000E6FF9EC0E6FF440EE66E9BC0E9FF9CC039
:102A3000EAFFEE52EF50E66E77EC12F0E552E55207
:102A4000E552E552F350DF6EDFCF10F01034E5525F
:102A5000E552E7CFD9FF1200D9CFE6FFE1CFD9FF8A
:102A6000020EE126010EDB6A7E0EE66EF0EC1FF030
:102A7000E552A850020BFDE06BD80009FAE1E66AC6
:102A8000F0EC1FF0E552A850020BFDE061D8000900
:102A9000FAE1FC0EDBCFE6FFF0EC1FF0E552A850A8
:102AA000020BFDE055D80009FAE1DF6AFC0EDB50AD
:102AB000DF5C2DE2DF50E76EFD0EDBCFE9FFFE0E9F
:102AC000DBCFEAFFE750E926000EEA22EF50E66E80
:102AD000F0EC1FF0E552DF50E76EFD0EDBCFE9FFB3
:102AE000FE0EDBCFEAFFE750E926000EEA22010ED8
:102AF000DBCFE7FFEF50E726010EE7CFDBFFA85063
:102B0000020BFDE025D80009FAE1DF2ACFD7010E3C
:102B1000DB28E86CE66EF0EC1FF0E552A8A2FED7C9
:102B2000020EE15C02E2E16AE552E16EE552E7CFB6
:102B3000D9FF1200D9CFE6FFE1CFD9FFFE0EDB505F
:102B400002E08A8201D08A92E552E7CFD9FF1200D3
:102B5000D9CFE6FFE1CFD9FFE6528150010BDF6EFE
:102B6000DF5002E0010E01D0000EE552E552E7CF42
:102B7000D9FF12008B8A12008B9A1200D9CFE6FF80
:102B8000E1CFD9FF020EE126FD0EDBCFE9FFFE0EFD
:102B9000DBCFEAFF030EE926000EEA22EFCFDFFFCC
:102BA000FD0EDBCFE9FFFE0EDBCFEAFF020EE926CA
:102BB000000EEA22010EEFCFDBFFFD0EDBCFE9FFB7
:102BC000FE0EDBCFEAFFEF50E66EFD0EDBCFE9FF36
:102BD000FE0EDBCFEAFF030EE926000EEA22E552E5
:102BE000E750EF6EFD0EDBCFE9FFFE0EDBCFEAFF15
:102BF000010EE926000EEA22EF50E66EFD0EDBCF55
:102C0000E9FFFE0EDBCFEAFF020EE926000EEA2204
:102C1000E552E750EF6EFD0EDBCFE9FFFE0EDBCF96
:102C2000EAFF010EE926000EEA22010EDBCFEFFFDC
:102C3000FD0EDBCFE9FFFE0EDBCFEAFFDFCFEFFFBC
:102C4000FD0EDBCFE9FFFE0EDBCFEAFF040EE92627
:102C5000000EEA22030EE926000EEA22EFCFDFFF84
:102C6000FD0EDBCFE9FFFE0EDBCFEAFF040EE92607
:102C7000000EEA22020EE926000EEA22010EEFCF34
:102C8000DBFFFD0EDBCFE9FFFE0EDBCFEAFF040E1C
:102C9000E926000EEA22EF50E66EFD0EDBCFE9FFDB
:102CA000FE0EDBCFEAFF040EE926000EEA22030E39
:102CB000E926000EEA22E552E750EF6EFD0EDBCF6B
:102CC000E9FFFE0EDBCFEAFF040EE926000EEA2242
:102CD000010EE926000EEA22EF50E66EFD0EDBCF74
:102CE000E9FFFE0EDBCFEAFF040EE926000EEA2222
:102CF000020EE926000EEA22E552E750EF6EFD0EC5
:102D0000DBCFE9FFFE0EDBCFEAFF040EE926000E63
:102D1000EA22010EE926000EEA22010EDBCFEFFFC8
:102D2000FD0EDBCFE9FFFE0EDBCFEAFF040EE92646
:102D3000000EEA22DFCFEFFF020EE15C02E2E16A61
:102D4000E552E16EE552E7CFD9FF1200D9CFE6FF99
:102D5000E1CFD9FFE652FD0EDBCFE9FFFE0EDBCF60
:102D6000EAFFEFCFDFFFFD0EDBCFE9FFFE0EDBCF8B
:102D7000EAFF010EE926000EEA22EF50E66EFD0E94
:102D8000DBCFE9FFFE0EDBCFEAFFE552E750EF6E47
:102D9000FD0EDBCFE9FFFE0EDBCFEAFF010EE926D9
:102DA000000EEA22DFCFEFFFE552E552E7CFD9FF71
:022DB00012000F
:0E2DB200D9CFE6FFE1CFD9FFFD0EDBCFFEF358
:102DC000FE0EDBCFFFF3FEC3E9FFFFC3EAFFEE6AAF
:102DD000ED6AFEC3E9FFFFC3EAFF020EEB6A030ED2
:102DE000EB6AFEC3E9FFFFC3EAFF040EEB6A050EC0
:102DF000EB6AFEC3E9FFFFC3EAFF060EE926000EF9
:102E0000EA22000EEE6E0C0EED6EE552E7CFD9FF12
:102E10001200D9CFE6FFE1CFD9FFFEC3E9FFFFC320
:102E2000EAFF040EE926000EEA22EECF10F0EFCF03
:102E300011F01E0ED8801056000E115610501110B1
:102E400004E1F6EC1CF0FF0E49D0FEC3E9FFFFC31E
:102E5000EAFF040EE926000EEA22EE2AED22FEC366
:102E6000E9FFFFC3EAFF060EE926000EEA22EECFD5
:102E700010F0EFCF11F0FEC3E9FFFFC3EAFF020E2F
:102E8000E926000EEA221050EE24E76E1150EE20E3
:102E9000EA6EE7CFE9FFFE0EDBCFEFFFFEC3E9FFEF
:102EA000FFC3EAFF020EE926000EEA22EE2AEF2215
:102EB000FEC3E9FFFFC3EAFF020EE926000EEA2285
:102EC0001E0EEE180AE1ED5008E1FEC3E9FFFFC354
:102ED000EAFF020EEB6A030EEB6A000EE552E7CF43
:102EE000D9FF1200D9CFE6FFE1CFD9FFE652FE0E9F
:102EF000DBCF10F0FEC3E9FFFFC3EAFF040EE926B3
:102F0000000EEA22EECF11F0EFCF12F01E0ED880A5
:102F10001156000E12561050115C000E125804E2A9
:102F2000F6EC1CF0FF0E64D0FE0EDB50106E116A42
:102F3000FEC3E9FFFFC3EAFF040EE926000EEA2202
:102F40001050EE261150ED22DF6AFE0EDB50DF5CE2
:102F50004EE2DF50E76EFC0EDBCFE9FFFD0EDBCF6C
:102F6000EAFFE750E926000EEA22EF50E66EFEC3C4
:102F7000E9FFFFC3EAFF060EE926000EEA22EECFC4
:102F800010F0EFCF11F0FEC3E9FFFFC3EAFF020E1E
:102F9000E926000EEA221050EE24E76E1150EE20D2
:102FA000EA6EE7CFE9FFE552E750EF6EFEC3E9FFB7
:102FB000FFC3EAFF020EE926000EEA22EE2AEF2204
:102FC000FEC3E9FFFFC3EAFF020EE926000EEA2274
:102FD0001E0EEE180AE1ED5008E1FEC3E9FFFFC343
:102FE000EAFF020EEB6A030EEB6ADF2AAED7000E91
:102FF000E552E552E7CFD9FF1200D9CFE6FFE1CF86
:10300000D9FFE652FE0EDBCF10F0FEC3E9FFFFC38F
:10301000EAFF040EE926000EEA22EECF11F0EFCF10
:1030200012F01050115C000E125804E2F6EC1CF085
:10303000FF0E57D0FE0EDB50106E116AFEC3E9FF83
:10304000FFC3EAFF040EE926000EEA221050EE5EEE
:103050001150ED5ADF6AFE0EDB50DF5C41E2FEC329
:10306000E9FFFFC3EAFF060EE926000EEA22EECFD3
:1030700010F0EFCF11F0FEC3E9FFFFC3EAFF1050DD
:10308000EE24E76E1150EE20EA6EE7CFE9FFEF5035
:10309000E66EDF50E76EFC0EDBCFE9FFFD0EDBCF07
:1030A000EAFFE750E926000EEA22E552E750EF6E0C
:1030B000FEC3E9FFFFC3EAFFEE2A000EEF22FEC3C4
:1030C000E9FFFFC3EAFF1E0EEE1808E1ED5006E12E
:1030D000FEC3E9FFFFC3EAFFEE6AED6ADF2ABBD752
:1030E000000EE552E552E7CFD9FF1200FEC3E9FF1B
:1030F000FFC3EAFF040EE926000EEA22EECF10F02D
:10310000EFCF11F01E0ED8801056000E115610C0D1
:08311000F3FF11C0F4FF1200EF
:08311800A58A9F86F1949F90A7
:103120009F92A292F190F09C9D86F2861200D08E22
:10313000F28EF28C1200F250800B800A01E0010E38
:10314000106E116A10BE116810C0F3FF11C0F4FFB9
:103150001200F250400B400A01E0010E106E116A9D
:1031600010BE116810C0F3FF11C0F4FF1200F2BCD2
:1031700004D0E1DFF350F41002E0F36A02D0010E54
:10318000F36EF46A1200F3DFF3CF10F0F4CF11F016
:10319000F350F41007E1CFDFF350F41003E1010E18
:1031A000F36E01D0F36AF46A1200DACFE4FFE2CFE3
:1031B000DAFFE9CFE4FFEACFE4FFF6CFE4FFF7CF91
:1031C000E4FFF8CFE4FFF5CFE4FFF3CFE4FFF4CF63
:1031D000E4FFFACFE4FFFBCFE4FF00EE00F0100EB7
:1031E000E80403E3EECFE4FFFBD700EE10F0040E9B
:1031F000E80403E3EECFE4FFFBD7E652A4AA03D032
:10320000E2EC1DF0A49A9EA603D098EC0AF09E96DC
:10321000E55200EE13F0040EE80403E3E5CFEDFF02
:10322000FBD700EE0FF0100EE80403E3E5CFEDFF4F
:10323000FBD7E5CFFBFFE5CFFAFFE5CFF4FFE5CF06
:10324000F3FFE5CFF5FFE5CFF8FFE5CFF7FFE5CFDB
:10325000F6FFE5CFEAFFE5CFE9FFE5CFDAFF1100A2
:10326000D8CFE4FFE0CFE4FFE46EDACFE4FFE2CFB3
:10327000DAFFE9CFE4FFEACFE4FFF6CFE4FFF7CFD0
:10328000E4FFF8CFE4FFF5CFE4FFF3CFE4FFF4CFA2
:10329000E4FFFACFE4FFFBCFE4FF00EE00F0100EF6
:1032A000E80403E3EECFE4FFFBD700EE10F0040EDA
:1032B000E80403E3EECFE4FFFBD7E652F0A004D02E
:1032C000F096EFEC1BF0F090F2A003D00DEC1CF0A8
:1032D000F290F2A403D06FEC1BF0F2949EA003D006
:1032E00088EC1BF09E909EA203D0ABEC1BF09E924C
:1032F000A1A203D0C4EC1BF0A192E55200EE13F0A2
:10330000040EE80403E3E5CFEDFFFBD700EE0FF07A
:10331000100EE80403E3E5CFEDFFFBD7E5CFFBFF9D
:10332000E5CFFAFFE5CFF4FFE5CFF3FFE5CFF5FFFB
:10333000E5CFF8FFE5CFF7FFE5CFF6FFE5CFEAFFF2
:10334000E5CFE9FFE5CFDAFFE550E5CFE0FFE5CFD8
:04335000D8FF100092
:0C335400929092929294929689908992A5
:10336000899489960101FE6BFF6BE66A0AD8E552E3
:10337000E66A07D8E55212008982000089920000AF
:103380001200D9CFE6FFE1CFD9FF020EE1268990E6
:10339000DE6ADD6ADECF10F0DDCF11F0D89011507B
:1033A00004E6080E105C000E115814E2FE0EDB500D
:1033B000010BE8B08984E8A08994DEDFFE0EDBCF44
:1033C000F3FFF390F342F3CFDBFFDF2A010EE2E3DA
:1033D000DB2AE0D78980020EE15C02E2E16AE55275
:1033E000E16EE552E7CFD9FF1200D9CFE6FFE1CF7A
:1033F000D9FFE652DF6A0101FE6BFF6B0A0E106E09
:103400000C6EFE0EDBCF07F076EC20F00350DF6E83
:10341000DF50090A34E0010A2DE00F0A26E0010A14
:1034200022E0030A1EE0010A17E0070A13E0010A7E
:103430000CE0030A07E0010A27E1700E0101FE1308
:103440000D0E21D00101FE8D13D0600E0101FE137F
:103450000E0E19D0600E14D0500E0101FE13030E93
:1034600012D0300E0DD0300E06D0700E0101FE13BA
:10347000FF810AD0700E0101FE130F0E04D0700EF2
:103480000101FE13070EFF130A0E106E0C6EFE0EE6
:10349000DBCF07F076EC20F00750DF6EDF50090A33
:1034A0002EE0010A27E00F0A20E0010A1CE0030ACF
:1034B00018E0010A14E0070A10E0010A09E0030A13
:1034C00004E0010A21E10D0E16D00101FE8710D0A3
:1034D0000E0E0101FE13C00E16D00E0E11D00B0EF3
:1034E00005D0070E0DD0070E06D00D0E0101FE13FC
:1034F000FF8B0AD00F0E0101FE13E00E04D00F0E59
:103500000101FE13600EFF130101FE51E66E39DF6B
:10351000E552000E0101FE15106EFF0EFF15116E33
:10352000106E116AE850E66E2CDFE552E552E55266
:10353000E7CFD9FF12000101FE51E66E22DFE5520E
:103540000101FF0EFF15106E116AE850E66E19DFDB
:04355000E55212002E
:0C35540029D8ADEF1AF0D9CFE6FFE1CF87
:10356000D9FF020EE126200EDF6EDE52270EDD6E41
:10357000D9CFE6FFDACFE6FF020EE66E180EE66E52
:10358000B1EC09F0E552E552E552E552DBEC0FF003
:103590000009FCE1020EE15C02E2E16AE552E16E43
:1035A000E552E7CFD9FF1200D9CFE6FFE1CFD9FF2F
:1035B000020EE126200EDF6EDE520F0EDD6ED9CF39
:1035C000E6FFDACFE6FF020EE66E690EE66EB1ECBC
:1035D00009F0E552E552E552E552DBEC0FF0000947
:1035E000FCE1020EE15C02E2E16AE552E16EE552C5
:1035F000E7CFD9FF1200D9CFE6FFE1CFD9FFE652DE
:10360000A80EDF6ED9CFE6FFDACFE6FF010EE66E39
:10361000180EE66EB1EC09F0E552E552E552E552BE
:10362000DBEC0FF00009FCE1060EE66E180EE66E0C
:1036300033EC0AF0E552E552DBEC0FF00009FCE157
:10364000E552E552E7CFD9FF1200D9CFE6FFE1CF2F
:10365000D9FFE652A80EDF6ED9CFE6FFDACFE6FF3C
:10366000010EE66E690EE66EB1EC09F0E552E55228
:10367000E552E552DBEC0FF00009FCE1060EE66EC8
:10368000690EE66E33EC0AF0E552E552DBEC0FF022
:0E3690000009FCE1E552E552E7CFD9FF120038
:02369E00970E85
:1036A000E66EA2EC1FF0E552D59E7B0EE66E830E11
:1036B000E66E0CEC1FF0E552E552CD900901FF6B70
:1036C000050EE66EBEEC1FF0E5527F0EE66E830E31
:1036D000E66E89EC1EF0E552E5527990120016D89C
:1036E000000EE66EE66A0A0EE66EE66A2EEC12F050
:1036F000E552E552E552E5521200000EE66EE66A2A
:1037000086EC1FF0E552E552D58E1200D59E1200D0
:103710000901FF2B030E106E0C6EFFC907F076EC4B
:1037200020F003500CE1000EE66EE66A0B0EE66E2A
:10373000E66A2EEC12F0E552E552E552E55212002F
:10374000000EE66EE66A6AEC1FF0E552E552CD80A7
:103750001200CD9012000901FF2B320EFF5D0EE129
:10376000FF6B10D8000EE66EE66A0C0EE66EE66A97
:103770002EEC12F0E552E552E552E5521200CC6A09
:10378000CA841200CA9412000401FE5108E1DBEC65
:103790001CF00401010EFE6FE66AEA0E06D0F4EC9E
:1037A0001CF00401FE6BE66A100EE66E4EEC1FF094
:1037B000E552E55212007980DBEC1CF00401010EA9
:1037C000FE6F12007990F4EC1CF00401FE6B120005
:1037D000928A94940E01020EE76FF19A1200000E85
:1037E000E66EE66A500EE66EE66A2EEC12F0E552E0
:1037F000E552E552E55212000A010F0EFE6FF19EEE
:103800009388938A938C938E8188818A818C818E10
:103810008A888A8A8A8C8A8E1200D9CFE6FFE1CF05
:10382000D9FFE652F00E8114E8380F0BDF6EDF503F
:103830000A01FE19010B13E0FEA105D0000EE66E91
:10384000E66A460E04D0000EE66EE66A470EE66EA5
:10385000E66A2EEC12F0E552E552E552E552DF50F1
:103860000A01FE19020B13E0FEA305D0000EE66E5E
:10387000E66A480E04D0000EE66EE66A490EE66E71
:10388000E66A2EEC12F0E552E552E552E552DF50C1
:103890000A01FE19040B13E0FEA505D0000EE66E2A
:1038A000E66A4A0E04D0000EE66EE66A4B0EE66E3D
:1038B000E66A2EEC12F0E552E552E552E552DF5091
:1038C0000A01FE19080B13E0FEA705D0000EE66EF4
:1038D000E66A4C0E04D0000EE66EE66A4D0EE66E09
:1038E000E66A2EEC12F0E552E552E552E552DFCFE2
:0C38F000FEFAE552E552E7CFD9FF1200C6
:0438FC001E0EF66E38
:10390000000EF76E000EF86E00010900F550966F7C
:103910000900F550976F03E1966701D03DD009008B
:10392000F550916F0900F550926F0900F550936FB3
:1039300009000900F550E96E0900F550EA6E09002A
:1039400009000900F550946F0900F550956F0900C2
:103950000900F6CF98F0F7CF99F0F8CF9AF091C020
:10396000F6FF92C0F7FF93C0F8FF0001945302E105
:10397000955307E00900F550EE6E9407F8E29507BD
:10398000F9D798C0F6FF99C0F7FF9AC0F8FF000179
:0A3990009607000E975BBFD71200E8
:06399A00949094929494B5
:1039A0008B908B928B940E010E0ED16F0F0ED26FF7
:1039B000120ED36F12003D0EE66E33EC20F0E5528E
:1039C000800EE66EE66A2DEC1EF0E552E5529EA2F0
:1039D000FED7FC0EE66E3F0EE66EB5EC1EF0E5522D
:1039E000E552BF80BF8212008DEF20F0E6681EEC2A
:1039F00020F0E552800EE66EE66AFEEC1DF0E55220
:103A0000E552B9800501010EFF6F12000AEC00F0CB
:103A10000501FF6B12000501FF5102E006EF1DF0EA
:043A2000F6EF1CF0B1
:0C3A2400D9CFE6FFDACFE6FFE1CFD9FFF3
:103A3000E2CFDAFFC26AC16AFC0EDB50400DF350E0
:103A4000C00B106EFC0EDB407F0B3C0B1010C26EE7
:103A5000FD0EDB50040DF350380B116EFD0EDB38FC
:103A60000F0B070B106EFD0EDB50800B10101110AA
:103A7000C16EFA0EDBCF10F0FB0EDBCF11F011C0E0
:103A800010F0116A10C048FFFA0EDBCF49FFFC0EA0
:103A9000DBAE03D09E9C9D8CF28CC280E552E5CFBC
:083AA000DAFFE7CFD9FF1200A5
:083AA800D9CFE6FFDACFE6FFFB
:103AB000E1CFD9FFE2CFDAFFA86A9C6AFD0EDBB046
:103AC000A888DBA202D0A88C9C8CDBB4A88EDBA6D5
:103AD00002D09C8801D09C8ADBA802D0A88401D0A7
:103AE000A894DBBA9C86DBAC02D0A38A01D0A39A4F
:103AF000DBAE02D0A38801D0A398FB0EDB50AB6EE7
:103B0000FC0EDBCF11F011C010F0116A10507D6E69
:103B1000A88A9C8EE552E5CFDAFFE7CFD9FF1200E5
:103B2000D9CFE6FFDACFE6FFE1CFD9FFE2CFDAFF68
:103B3000AD6AAC6AFD0EDBB0AD88DBA202D0AD8C05
:103B4000AC8CDBB4AD8EDBA602D0AC8801D0AC8AE5
:103B5000DBB8AD84DBBAAC86DBAC02D09D8A01D089
:103B60009D9ADBAE02D09D8801D09D98FB0EDB5064
:103B7000B06EFC0EDBCF11F011C010F0116A1050C6
:103B80007F6EAD8AAC8EE552E5CFDAFFE7CFD9FF85
:023B9000120021
:0E3B9200400EE66EE66A3C0EE66E90EC1DF00C
:103BA000E552E552E5520E01050EF66FCC6F400E60
:103BB000E66EE66A7C0EE66E54EC1DF0E552E552C8
:103BC000E5521200A4AA06D02FEC1FF0E66EF0EC2E
:103BD00013F0E5520901FEA710D0AC98AC889C9870
:103BE0009C88000EE66EE66A1E0EE66EE66A77ECCC
:0C3BF00012F0E552E552E552E5521200D9
:043BFC00D9CFE6FF38
:103C0000DACFE6FFE1CFD9FFE2CFDAFFE652E652A4
:103C1000FC0EDBCF10F0FD0EDBCF11F0060ED890BE
:103C200010361136E804FBE110C0DEFF11C0DDFFE5
:103C3000010EDB50B56EDF50E840E8403F0B300B23
:103C4000106ECF0EB4141010B46EE552E552E5526A
:0A3C5000E5CFDAFFE7CFD9FF12003D
:063C5A00D9CFE6FFDACF2E
:103C6000E6FFE1CFD9FFE2CFDAFFE652E652FC0EE3
:103C7000DBCF10F0FD0EDBCF11F0060ED890103622
:103C80001136E804FBE110C0DEFF11C0DDFF010EBC
:103C9000DB50BB6EDF50E840E8403F0B300B106E4E
:103CA000CF0EBA141010BA6EE552E552E552E5CFC8
:083CB000DAFFE7CFD9FF120093
:083CB8009280FE0EE66E1F0E65
:103CC000E66E840EE66EE10EE66E12EC1DF0E55235
:103CD000E552E552E55212008FEF20F007EF00F0B9
:103CE000D9CFE6FFE1CFD9FF030EE12684EC20F027
:103CF000F3CFDEFFF4CFDDFF020EF36EDB6E030EBB
:103D0000E15C02E2E16AE552E16EE552E7CFD9FFFC
:023D100012009F
:0E3D1200D9CFE6FFDACFE6FFE1CFD9FFE2CF4F
:103D2000DAFFFC0EDB50F30B976EFD0EDB507F0BC2
:103D3000E824796EFD0EDBB4CD867B6A7A6AA192A7
:103D4000A492DBAE02D0A08201D0A092FC0EDBA434
:103D500002D0A38201D0A39297BE97867980E552C4
:0A3D6000E5CFDAFFE7CFD9FF12002C
:063D6A00D9CFE6FFDACF1D
:103D7000E6FFE1CFD9FFE2CFDAFFFD0EDB80DB8289
:103D8000DB84DB86DB88DB8AFC0EDB84DB86DB887E
:103D9000DB8ADB8CDB8EFD0EDBCFE6FFC00EBA10BC
:103DA000E552E714BA6EFC0EDBCFE6FF0F0EBA1039
:103DB000E552E714BA6EE552E5CFDAFFE7CFD9FF57
:023DC0001200EF
:0E3DC200D9CFE6FFDACFE6FFFA0EE3CFD9FF46
:103DD000FB0EE3CFDAFFFC0EE3CFE9FFFD0EE3CFEE
:103DE000EAFFE9CFF3FFEACFF4FFF80EE35003E177
:103DF000F90EE35008E0F80EE30602E2F90EE306DE
:103E0000DECFEEFFF2D7FF0EE3CFDAFFE552FF0E73
:083E1000E3CFD9FFE5521200D7
:083E1800D9CFE6FFDACFE6FF87
:103E2000E1CFD9FFE2CFDAFFFC0EDB50F30B9A6E45
:103E3000FD0EDB507F0BE824CD6ECF6ACE6A9E90DC
:103E4000FD0EDBAE02D09D8001D09D909ABE9A8679
:0E3E5000CD80E552E5CFDAFFE7CFD9FF1200B3
:023E5E00D9CFBA
:103E6000E6FFDACFE6FFE1CFD9FFE2CFDAFFE65295
:103E7000F20E0901FE179CAC03D0FE919CB0FE81AE
:103E80009CB4FE859CB2FE87AA50DF6EDF50E552DF
:0C3E9000E552E5CFDAFFE7CFD9FF1200C2
:043E9C00D9CFE6FF95
:103EA000DACFE6FFE1CFD9FFE2CFDAFFE652E65202
:103EB000FC0EDBCFDEFFDBCFDDFF010EDB507B6EC8
:103EC000DF507A6EE552E552E552E5CFDAFFE7CFF3
:043ED000D9FF120004
:0C3ED400D9CFE6FFDACFE6FFE1CFD9FF3F
:103EE000E2CFDAFFE652E652FC0EDBCFDEFFDBCF9D
:103EF000DDFF010EDB50CF6EDF50CE6EE552E55296
:0C3F0000E552E5CFDAFFE7CFD9FF120051
:043F0C00D9CFE6FF24
:103F1000DACFE6FFE1CFD9FFE2CFDAFFE652E65291
:103F2000FC0EDBCFDEFFDBCFDDFF010EDB50D76EFB
:103F3000DF50D66EE552E552E552E5CFDAFFE7CF26
:043F4000D9FF120093
:0C3F4400D9CFE6FFDACFE6FFE1CFD9FFCE
:103F5000E2CFDAFFFD0EDB507F0BD56ED76AD66A53
:103F6000F294FD0EDBAE02D0F28A01D0F29AD58E29
:0C3F7000E552E5CFDAFFE7CFD9FF1200E1
:043F7C00D9CFE6FFB4
:103F8000DACFE6FFE1CFD9FFE2CFDAFFFD0EDB505B
:103F9000FB0BCA6ECC6A9E92FD0EDBAE02D09D82F8
:103FA00001D09D92CA84E552E5CFDAFFE7CFD9FF71
:023FB0001200FD
:0E3FB200FF0EE350156EEF0E01D0F30EE76E1A
:103FC000E72EE0EF1FF00C0E146EE76AE72EE6EF27
:103FD0001FF0142EE5EF1FF0152EDEEF1FF012007C
:103FE000D9CFE6FFDACFE6FFE1CFD9FFE2CFDAFFA4
:103FF000A8AC04D0A8900901FEB3A880FD0EDB5048
:0E400000A96EE552E5CFDAFFE7CFD9FF120037
:02400E007DEF44
:104010001BF0E66AC1EC19F0E552E66AC1EC19F052
:10402000E552BAEF15F0BCEC15F0020EE66ED9ECD5
:0C4030001FF0E5529BEC1AF086EF1BF02D
:04403C00D9CFE6FFF3
:10404000DACFE6FFE1CFD9FFE2CFDAFF0C0EB46E94
:10405000CA94FD0EDB50CB6ECA84E552E5CFDAFF81
:06406000E7CFD9FF1200BA
:0A406600D9CFE6FFDACFE6FFE1CF85
:10407000D9FFE2CFDAFF0C0EBA12CA94FD0EDB5064
:10408000CB6ECA84E552E5CFDAFFE7CFD9FF120045
:10409000FF0EE350156E480E01D04C0EE76EE72E72
:1040A000FED7E76AE72EFED7152EF7D700001200DD
:1040B000C00EF36E00EE00F00E0E01D81200EA60A2
:1040C00002D0EE6AFCD7F350E9601200EE6AFCD72A
:1040D0001EEE00F02EEE00F0F86A0F9C7EEC1CF055
:0C40E00003EC00F02EEC00F0FBD7120007
:0440EC00036A080E4D
:1040F000E76ED890073603360C50035C02E3036E7C
:08410000072AE72EF7D7120091
:08410800C450136E126AC3508B
:0A4110001210F36E13C0F4FF12004A
:04411A00BA6A12006B
:02411E00C2825B
:0241200012008B
:0241220000009B
:02412400000099
:02412600000097
:02412800000095
:02412A00000093
:01FFF800A068
:01FFFA00DD29
:01FFFD00F80B
:00000001FF
